:1000000000308A0004280000FF238316900000308F
:100010008A00752883161F080F3930389F00831215
:100020001F080C3981389F0083161F08F0390138EA
:100030009F0083121F1385282C30840000080319A9
:1000400030280130A100A001A00B2428A10B2328F7
:100050004A30A000A00B2A2800000000800B2128B5
:100060000034A808031D3628851237288516003469
:10007000280DA000A00DFC30A0051F08C3392004E6
:100080009F00AA01A901AB012B08073C031C5828BB
:100090009F149F18492883161E088312A907031866
:1000A000AA0A1E08AA070230AC001C20AB0A44288A
:1000B000AA0CA90CAA0CA90CAA0CA90C1F30AA0501
:1000C0002908A1002A08A200A928003085190130BA
:1000D000003A031D7028F330A1000230A2007428FA
:1000E0004330A1000330A200AE2884011F308305F5
:1000F00083161F08F0399F0083121F1307309F00DB
:100100005A30A6000F3065000A2856308316810049
:10011000063095008312A7012708093C031C9A2882
:100120000516C830AC001C200512C830AC001C20DD
:10013000A70A8C280130A8003120003005190130B1
:10014000003A031DA7280130A8003120C828A801C3
:1001500038282208A9002108A800652829082202B9
:10016000031CC228031DB828210828020318C2282E
:10017000A608031DBF28A80131200512C128A60327
:100180000516C8280130A800312005125A30A600F3
:100190002830A800FA30AC001C20A80BCA289D28E3
:0201A0006300FA
:02400E00C439B3
:00000001FF
